:1000000008308A00612A00000A108A100A1182074B
:100010004E344134523444345334203468346134DF
:1000200000340A108A100A11820766346934723467
:100030007334743443346834613472344F34663406
:100040002034463469346C34653420344E346134A1
:100050006D3465342034693473343A34253458347B
:1000600000340A108A100A11820774346834693423
:100070007334203473346F346E3467342034733403
:1000800074346134723474347334203461347434AD
:1000900020343A34253434344C3458342034003449
:1000A0000A108A100A1182077434683465342034C7
:1000B000623470346234733474346134723474343E
:1000C0002034253438344C3458342034203400342F
:1000D0000A108A100A118207743468346534203497
:1000E0004234503442345F3462347934743473347B
:1000F0007034653472347334653463342034253499
:1001000038344C3458342034203400340A108A10E7
:100110000A11820774346834653420344234503410
:1001200042345F345334653463345034653472344C
:1001300043346C34753473342034253438344C34BF
:1001400058342034203400340A108A100A118207EF
:1001500074346834653420344234503442345F346B
:1001600052346534733476346434533465346334D0
:1001700043346E3474342034253438344C34583499
:100180002034203400340A108A100A118207743493
:100190006834653420344234503442345F344E3451
:1001A00075346D344634413454347334203425343A
:1001B00038344C3458342034203400340A108A1037
:1001C0000A11820774346834653420344234503460
:1001D00042345F3452346F346F34743445346E3487
:1001E000743443346E3474342034253438344C340D
:1001F00058342034203400340A148A100A1182073B
:1002000074346834653420344234503442345F34BA
:1002100046344134543453347A343134363420340F
:10022000253438344C3458342034203400340A1403
:100230008A100A11820774346834653420346634B5
:1002400061347434733474346134723474342034EB
:10025000253438344C3458342034203400340A14D3
:100260008A100A11820774346834653420344634A5
:10027000693472347334743452346F346F34743478
:100280004434693472345334653463344E347534D1
:100290006D342034253438344C34583420342034F0
:1002A00000340A148A100A118207743468346534E1
:1002B00020344634693472347334743444346134D1
:1002C0007434613453346534633474346F34723449
:1002D0002034253438344C3458342034203400341D
:1002E0000A148A100A118207743468346534203481
:1002F00052346F346F347434443469347234533448
:100300006534633474346F34723473342034253478
:1003100038344C345834203420340034F9308316C7
:100320008600831206110330F700F70B9529061596
:1003300000340711610893000330F700F70B9E2982
:1003400000000000620893000330F700F70BA629B5
:1003500000000000630893000330F700F70BAE299C
:1003600000000000663084001308800064089300D9
:100370000330F700F70BBA29000000006530840055
:10038000130880000730F700F70BC42900000000B5
:1003900007156508F8006608F9000034F93083167F
:1003A0008600D2308700223085008801890106301E
:1003B0009F00810183129F01071518308500890174
:1003C0008E219817831699011816181398179816E6
:1003D0001417831294160230E1000B30E200203033
:1003E000E3002030E40099218A150A126C2A61305A
:1003F0008400000803190B2A0130F800F701F70BFD
:10040000FF29F80BFE294A30F700F70B052A0000F8
:100410000000800BFC29003486140830F80000002E
:1004200000000000F817242AF813D70C03188610D0
:10043000031C86147817242A7813F80B152A000059
:10044000000000008610242A0B308400840B262A2A
:10045000F81B142A781B1C2A0034851E2D2A003410
:100460002D22FF3083168800831288018511080829
:10047000A00085152D2285110808A1008515831679
:100480008801831200348518432A051500000000F6
:1004900005116430E100F72107308900EC30880055
:1004A0002D220512051630228A150A129A2A0F30BB
:1004B000EB05E030EB046B30840000088800063068
:1004C0008900051205166A3084000008880005308E
:1004D0008900051205166930840000088800043080
:1004E0008900051205166830840000088800033072
:1004F00089000512051601308800023089000512B6
:10050000051620308800073089000512051689017C
:100510000034E8080319962A851E8C2A8511851552
:10052000851E902A85118515E803892A0034F80173
:10053000F901F701FA015408031DA12A5308031910
:10054000BB2A1030D5000310D10DD20DF70DFA0DD6
:1005500054087A02031DAE2A53087702031CB72AF7
:100560005308F702031CFA035408FA020314F80DA7
:10057000F90DD50BA32A00008A110A12872B10301F
:10058000F700FA01D301D00CCF0C031CCD2A51087F
:10059000FA070318D30A5208D307D30CFA0CF90C44
:1005A000F80CF70BC32A0034D61BE62A0F30F700ED
:1005B000550EF7050A3077020318E12A3030F707A5
:1005C000E32A5608F7077708D7000C220F30D50525
:1005D0000A3055020318EE2A3030F02AD613560896
:1005E000D5075508D7000C220034EB01EA01E901D8
:1005F000E8015722E330E80089223022CE012108A9
:10060000CD00A500A4012008A4070318A50AD00165
:10061000CF012508CE002408CD005008EB004F087C
:10062000EA004E08E9004D08E80057220530E800CE
:1006300089223022C3012108C2003022CE012008C5
:10064000CD00FA000030C2070318C30A7A08C307B6
:100650002108A2003022CE012108CD00D000CF0118
:1006600020084F07AA005008AB000318AB0A30223D
:100670002008C800C5012108C4003022CE0120088E
:10068000CD00FA000030C4070318C50A7A08C50770
:1006900030223022CE012108CD00FA0000302007A0
:1006A000C6007A08C7000318C70A2A082407AC0046
:1006B0002508AD000318AD0A2B08AD07440DCD0089
:1006C000450DCE00CD0DCE0DCD0DCE0DCD0DCE0DEB
:1006D000CD0DCE0DE030CD0501304202F7004308CC
:1006E000FA000030031C0130FA0277084D07CF00F2
:1006F0004E08D0000318D00A7A08D0075008D2005C
:100700004F08D1004308D4004208D300972A790843
:10071000A7007808A600D0014808CF004708D200FB
:100720004608D100BF227908FA0078082A07CD00D0
:100730002B08CE000318CE0A7A08CE0726084D07EC
:10074000A8004E08A9000318A90A2708A907CE0186
:100750004808CD004E08D0004D08CF004708D20011
:100760004608D100BF227908FA0078082A07B200AB
:100770002B08B3007A0803187A0FB307B401B50148
:100780000D30D7000C220A30D7000C22CD014D08C5
:100790005020CD0AD7000C220C304D02031DC72B70
:1007A0000530CE003A30D7000C22CE0BD22B2030B1
:1007B000D7000C220430CF003030D7000C22CF0BF2
:1007C000DC2B2508D5003730D600D4222408D500EC
:1007D0003730D600D4222030D7000C222030D7006A
:1007E0000C220D30D7000C220A30D7000C220D301D
:1007F000D7000C220A30D7000C22CD014D0868200A
:10080000CD0AD7000C2212304D02031DFE2B0530FD
:10081000CE003A30D7000C22CE0B092C2030D70066
:100820000C220430CF003030D7000C22CF0B132C19
:100830004308D5003730D600D4224208D5003730DF
:10084000D600D4222030D7000C222030D7000C2232
:100850000D30D7000C220A30D7000C22CD014D08F4
:100860008620CD0AD7000C2212304D02031D2F2CFA
:100870000530CE003A30D7000C22CE0B3A2C203077
:10088000D7000C220430CF003030D7000C22CF0B21
:10089000442C2208D5003730D600D4222030D7008F
:1008A0000C222030D7000C220D30D7000C220A3049
:1008B000D7000C22CD014D08A420CD0AD7000C2270
:1008C00013304D02031D5B2C0530CE003A30D700AB
:1008D0000C22CE0B662C2030D7000C220430CF0027
:1008E0003030D7000C22CF0B702C2B08D5003730BE
:1008F000D600D4222A08D5003730D600D4222030A2
:10090000D7000C222030D7000C220D30D7000C224B
:100910000A30D7000C22CD014D08C320CD0AD700E4
:100920000C220F304D02031D8C2C0530CE003A30C6
:10093000D7000C22CE0B972C2030D7000C2204308D
:10094000CF003030D7000C22CF0BA12C4808D500A7
:100950003730D600D4222030D7000C222030D700E8
:100960000C220D30D7000C220A30D7000C22CD010A
:100970004D08DE20CD0AD7000C2212304D02031D97
:10098000B82C0530CE003A30D7000C22CE0BC32C49
:100990002030D7000C220430CF003030D7000C229A
:1009A000CF0BCD2C4508D5003730D600D4224408D3
:1009B000D5003730D600D4222030D7000C2220308A
:1009C000D7000C220D30D7000C220A30D7000C22A1
:1009D000CD014D08FC20CD0AD7000C220F304D026E
:1009E000031DE92C0530CE003A30D7000C22CE0B87
:1009F000F42C2030D7000C220430CF003030D70048
:100A00000C22CF0BFE2C4708D5003730D600D4225D
:100A10004608D5003730D600D4222030D7000C222B
:100A20002030D7000C220D30D7000C220A30D7001E
:100A30000C220D30D7000C220A30D7000C22CD0139
:100A40004D081721CD0AD7000C220C304D02031D92
:100A5000202D0530CE003A30D7000C22CE0B2B2DA6
:100A60002030D7000C220430CF003030D7000C22C9
:100A7000CF0B352D2D08D5003730D600D4222C08C9
:100A8000D5003730D600D4222030D7000C222030B9
:100A9000D7000C220D30D7000C220A30D7000C22D0
:100AA000CD014D082F21CD0AD7000C2216304D0262
:100AB000031D512D0530CE003A30D7000C22CE0B4D
:100AC0005C2D2030D7000C220430CF003030D7000E
:100AD0000C22CF0B662D3508D5003730D600D42236
:100AE0003408D5003730D600D4223308D50037304B
:100AF000D600D4223208D5003730D600D422203098
:100B0000D7000C222030D7000C220D30D7000C2249
:100B10000A30D7000C22CD014D085121CD0AD70053
:100B20000C2213304D02031D8C2D0530CE003A30BF
:100B3000D7000C22CE0B972D2030D7000C2204308A
:100B4000CF003030D7000C22CF0BA12D2908D500C3
:100B50003730D600D4222808D5003730D600D4222A
:100B60002030D7000C222030D7000C220D30D700C7
:100B70000C220A30D7000C22CD014D087021CD0A7D
:100B8000D7000C2212304D02031DBD2D0530CE00C2
:100B90003A30D7000C22CE0BC82D2030D7000C22C3
:100BA0000430CF003030D7000C22CF0BD22D2708D5
:100BB000D5003730D600D4222608D5003730D600ED
:100BC000D4222030D7000C222030D7000C220D3048
:100BD000D7000C220A30D7000C220D30D7000C228F
:100BE0000A30D7000C228A150A129D2A871C0D2E66
:100BF000E201E1016208073C031C0D2EE30107142A
:100C000063089900000000000710000000000000C9
:100C10000000E10A0319E20AFA2D00340230E10073
:100C2000E2010330E3000430E40099210230E100E6
:100C3000E2010330E300E4019921F625003420307D
:100C4000F100ED01EE01EF01F0016808FA0067081C
:100C5000F9006608F8006508F7000310771C3E2EBF
:100C60006908ED076A0803186A0FEE076B08031896
:100C70006B0FEF076C0803186C0FF007F00CEF0C0C
:100C8000EE0CED0CFA0CF90CF80CF70CF10B2D2E08
:100C900000344E0CFA004D0CF900FA0CF90CFA0C69
:100CA000F90CFA0CF90C0F30FA0579083207D30069
:100CB0003308D4007A0803187A0FD4073408D50013
:100CC000003003180130D5073508D600003003186E
:100CD0000130D60724085307D7005408D800250848
:100CE0000318250FD8075508D90000300318013024
:100CF000D9075608DA00003003180130DA075A081D
:100D0000EB005908EA005808E9005708E8005722A4
:100D10004D080F39D3004E080039D400530DD500CB
:100D2000540DD600D50DD60DD50DD60DD50DD60D3D
:100D3000F030D5055508E80089223022D301530848
:100D40001120D30AD7000C2219305302031D9F2E05
:100D50002008D5003730D600D4220330D40020300C
:100D6000D7000C22D40BAF2EA008031DBA2E0230E0
:100D7000F800D02F2008E53C0319CE2FFE30D70015
:100D80000C220130D7000C222008D7000C222108A9
:100D9000D7000C2230222008D7000C222108D700CF
:100DA0000C2230222008D7000C222108D7000C2268
:100DB00030222008D7000C222108D7000C222E3028
:100DC000D7000C2230222008D7000C222108D7009F
:100DD0000C222008D0002108D10030222008D700A2
:100DE0000C222108D7000C220D30D7000C220A302B
:100DF000D7000C222008D20050086D3C0319042FA4
:100E000050084D3C031DCE2F5108503C03190C2FA8
:100E10005108703C031DCE2F5208333C031DCE2FCA
:100E20000730E80089223022D4012108D300D600FF
:100E3000D50120085507AE005608AF000318AF0AC9
:100E4000D30153083120D30AD7000C2215305302A6
:100E5000031D212F0330D4002030D7000C22D40BE7
:100E60002C2F2F08D5003730D600D4222E08D500DD
:100E70003730D600D4222030D7000C22D601D5013D
:100E8000D4012008D300DA01D901D8012108D70004
:100E90005908FA005808F9005708F800F7017708D0
:100EA0005307DC005408DD0078080318780FDD07CD
:100EB0005508DE0079080318790FDE075608DF00B1
:100EC0007A0803187A0FDF0702305C02E0005D0841
:100ED000E1000030031C0130E1025E08E200003056
:100EE000031C0130E2025F08E3000030031C013004
:100EF000E3026308E8006208E7006108E6006008B2
:100F0000E500EC01EB01EA012208E9001F267A085E
:100F1000E4007908E3007808E2007708E10024089B
:100F20006107E5006208E60025080318250FE607BB
:100F30006308E700003003180130E7076408E800A1
:100F4000003003180130E80728086507B600660876
:100F5000B70029080318290FB7076708B800003041
:100F600003180130B8076808B900003003180130D1
:100F7000B90730223A308400200880003B308400DA
:100F80002108800030223C308400200880003D3061
:100F90008400210880000130F800D02F0030F800D4
:020FA00000341B
:10100000F701F801F901FA01E901EA01EB01EC014C
:10101000680867046604650403193E282030ED0063
:101020000310E10DE20DE30DE40DE90DEA0DEB0D0A
:10103000EC0D68086C02031D272867086B02031D6E
:10104000272866086A02031D272865086902031C11
:1010500038286508E9026608031C660FEA0267087B
:10106000031C670FEB026808031C680FEC020314F3
:10107000F70DF80DF90DFA0DED0B10280000693091
:1010800084000034E001DE018A110E268A1554081E
:10109000E4005308E3005208E2005108E100E801CF
:1010A000E701E6012208E50000207A08D40079086B
:1010B000D3007808D2007708D1005808E400570818
:1010C000E3005608E2005508E100E801E701E60107
:1010D0002208E50000207A08D8007908D7007808AF
:1010E000D6007708D50054085802031C5C2A031D5B
:1010F000892853085702031C5C2A031D89285208BB
:101100005602031C5C2A031D892851085502031C42
:101110005C2AE0012208600203186A2902302E02CC
:10112000D9002F08DA000030031C0130DA02DB019D
:10113000DC012208F700F801F901FA017A08E4005D
:101140007908E3007808E2007708E1005C08E8002D
:101150005B08E7005A08E6005908E5006408EC005F
:101160006308EB006208EA006108E9008A111F26A3
:101170008A157A08DC007908DB007808DA0077083D
:10118000D9002408F7002508F800F901FA017708CA
:10119000D90778080318780FDA0779080318790F48
:1011A000DB077A0803187A0FDC072808F7002908FC
:1011B000F800F901FA017708D90778080318780FC1
:1011C000DA0779080318790FDB077A0803187A0F12
:1011D000DC076008F700F801F901FA017708D90780
:1011E00078080318780FDA0779080318790FDB07F6
:1011F0007A0803187A0FDC075C08EB005B08EA004A
:101200005A08E9005908E8008A1157228A15631420
:10121000FF308316880010308312E200E2080319C1
:10122000342987181529631011291030E100E108CD
:10123000031932298A112D228A15851107140808ED
:101240009900851507100000000000000000000054
:101250008511071408089900851507100000000083
:10126000E1031729E2030E29831688010030831257
:1012700063180130F800F80803196129DE0A5E08D6
:10128000783C031860290330E1000B30E200E301F1
:10129000E4018A1199218A157808C9008A118E21E2
:1012A0008A158A110E268A150230E1000B30E20001
:1012B0004908E3004908E4008A1199218A15DE01F2
:1012C0006829DE035E08013C031C68290230DE0049
:1012D000E00A8A282F08B1002E08B000E401E301DB
:1012E0003108E2003008E100613084000008E700C6
:1012F0006208E1006308E2006408E300E4012C08EE
:10130000E1072D0803182D0FE20700300318013004
:10131000E307003003180130E4076408EB006308BA
:10132000EA006208E9006108E8008A1157228A157C
:101330006708E8008A1189228A158A1130228A15E5
:10134000E9012108E800EB00EA01FA0120086A0738
:10135000E5006B08E6000318E60A7A08E607650868
:10136000F8006608F9007908AF007808AE00861921
:101370000E2A5D10FA30DF000330E1000B30E2008E
:101380000330E3001430E4008A1199218A157808AB
:10139000C9008619D7290830E1008A11F7218A157A
:1013A000DF08031DD52906115D14DF03C9290830A4
:1013B0008B0063008B015D1C0B2A06150130E100D8
:1013C0008A11F7218A150230E100E2010330E300BF
:1013D0000430E4008A1199218A150130E1008A1154
:1013E000F7218A150230E100E2010330E300E40155
:1013F0008A1199218A150130E1008A11F7218A1595
:101400000230E1000B30E2004908E3004908E40043
:101410008A1199218A158A11F6258A15861A2A2A8F
:101420000330E1000B30E200E301E4018A1199216D
:101430008A157808C900490F1E2A1F2AC90A0230D6
:10144000E1000B30E2004908E3004908E4008A119A
:1014500099218A15061A462A0330E1000B30E20072
:10146000E301E4018A1199218A157808C900C908A5
:1014700003193B2AC9030230E1000B30E20049089E
:10148000E3004908E4008A1199218A15861B4B2A3A
:101490006E30F8005E2A061B532AA3080319532A4C
:1014A0007030F8005E2A0130D1070318D20A031900
:1014B000D30A0319D40A73287330F8008A150A1264
:1014C000F72A84011F3083050F3083169F00831293
:1014D0008610C9018A11CE298A15FF30E1008A11D0
:1014E000F7218A15FF30E1008A11F7218A15FF30B4
:1014F000E1008A11F7218A15FF30E1008A11F721F6
:101500008A150330CD002030D7008A110C228A15AD
:10151000CD0B832ACE014E088A1104208A15CE0AEB
:10152000D7008A110C228A1508304E02031D8B2A1F
:101530008A11432A8A158A11F52A8A158A110E26DC
:101540008A150230E1000B30E2002030E300203049
:10155000E4008A1199218A150130A3007330CC0070
:10156000861F072B061F072BCE012308CD008A11EB
:1015700049268A157808023C031DC22A0130A300BF
:101580007330CC00CE012308CD008A1149268A157C
:10159000780BF92A0310FA013D0CF9003C0CF80015
:1015A0003B0CF7003607CD003708CE00780803184B
:1015B000780FCE073808CF0079080318790FCF07C6
:1015C0003908D0007A0803187A0FD0073908D400F8
:1015D0003808D3003708D2003608D1005008D800A8
:1015E0004F08D7004E08D6004D08D500422878088D
:1015F000CC004C086E3C0319012B4C08733C031DB6
:10160000022BA30A4C08703C031D072BA303B02A2E
:02161000630075
:02400E00FA3F77
:00000001FF
